:020000040000FA
:1000000083161C308500023086008312850186012C
:10001000FF309F008B018C2E7930A0001430A1009E
:10002000A00B1028A10B10288613061186110616A6
:1000300086122E205130A0000630A100A00B1E28F1
:10004000A10B1E282B302B2013302B200C302B2003
:1000500004302B20080086133120080006170613F1
:100060000800A0000615861506168616A01F0611A4
:10007000201F8611A01E0612201E86122E20061595
:10008000861506168616A01D0611201D8611A01CB9
:100090000612201C86122E2086172130A000A00BED
:1000A0004F2808000130861331209730A00003301C
:1000B000A100A00B5928A10B5928803086133120AC
:1000C0000800861331200800A00003112008003A20
:1000D000031930342008013A031931342008023A58
:1000E000031932342008033A031933342008043A40
:1000F000031934342008053A031935342008063A28
:10010000031936342008073A031937342008083A0F
:10011000031938342008093A03193934403452207D
:10012000483031206530312061303120BA30312003
:10013000BF303120B8303120B3303120B8303120D9
:10014000703031206F303120B330312061303120B8
:10015000BD3031206F30312021303120C03061205E
:10016000613031206D303120703031202D30312020
:100170007230312075303120403031206D303120E7
:1001800061303120693031206C3031202E30312007
:10019000723031207530312008005220A1303120DA
:1001A000703031206F303120BC303120BA303120F6
:1001B0006F30312063303120BF303120C4303120E6
:1001C000080052205430312065303120BC303120BD
:1001D000B23031207030312020303120080086309C
:1001E0006120BD303120B8303120B7303120BA30F5
:1001F0003120B83031206530312008008630612050
:10020000B3303120C3303120633031206F303120A2
:10021000BA303120B830312065303120080052200A
:10022000A030312061303120BB30312061303120AD
:10023000BD3031206330312020303120080087303C
:100240006120BE3031206530312070303120653082
:100250003120E3303120BD303120B83031206530DD
:100260003120080087306120B730312061303120E3
:10027000E3303120BD303120B830312065303120BD
:1002800008005220E130312065303120BD3031206E
:10029000BF303120703031206F303120B330312009
:1002A000BA303120613031200800522042303120F4
:1002B000C3303120B23031206F30312070303120E6
:1002C00020303120B3303120783031206F30312070
:1002D000E33031206130312008005220A430312039
:1002E000B330312079303120BA3031202030312004
:1002F000080085306120B3303120BA303120BB3066
:100300003120C6303120C030312065303120BD3041
:100310003120080085306120B3303120C3303120D6
:10032000BA303120BB303120C6303120C0303120CE
:1003300065303120BD30312008005220423031205C
:100340007030312065303120BC303120C730312051
:1003500020303120B830312020303120E3303120BE
:1003600061303120BF303120613031200800C03091
:100370006120483031206130312063303120BF307E
:100380003120703031206F303120B8303120BF3013
:100390003120C43031203F303120CB306120080083
:1003A000E330312061303120203031200800BD3071
:1003B000312065303120BF303120080052205430C8
:1003C000312065303120BC303120BE3031206530E5
:1003D00031207030312061303120BF303120793010
:1003E00031207030312061303120BF306120423007
:1003F000312065303120BD303120BF303120B83060
:100400003120BB303120C7303120BF3031206F3038
:100410003120703031200800522041303120BA3074
:100420003120BF303120B8303120B330312061303D
:100430003120E5303120B8303120C7303120203034
:100440003120763031202E30312033303120E330EE
:10045000312008005220843061204F303120B630E6
:100460003120B8303120E330312061303120BD30CF
:100470003120B83031206530312008000514851452
:100480004A2205104A22851008004A2285144A2271
:100490000514080000000800A0007F220830A10019
:1004A00056224A2285144A2285100800A00D051004
:1004B0000318051485144A228510A10B562A08003A
:1004C0007B220830A1008514031005180314A00D29
:1004D00085104A22A10B632A08007F22051085148B
:1004E0004A228510200808007F22051485144A221C
:1004F000851020080800831605148312080083164F
:10050000051083120800A0007F220830A1003E22BF
:1005100056227B224A222712051C271674224522C6
:10052000080003113C08643A0319BC03A92A03110B
:100530003C08413A0319BC03A92A03113C08113AAB
:100540000319BC03A92A03113C08043A0319BC038C
:10055000A92A3C08FF3A0319BC0A0800031128081D
:100560000A3A0319A803D22A03112808183A0319D2
:10057000A803D22A031128083C3A0319A803D22A57
:1005800003112808203A0319A803D82A03112808C0
:100590000D3A0319A803D82A03112808643A03194D
:1005A000A803D22A03112808FF3A0319A80A080051
:1005B00003112808003A0319A80A080003113C088F
:1005C000113A0319BC033C08003A0319BC0A08009D
:1005D0003C08A000A601A501A40103146430A002F8
:1005E000031CF42AA60AEE2AA0070A30A002031C64
:1005F000FB2AA50AF52A2007A40008002608642083
:10060000312025086420312024086420312008008E
:10061000AD30A4001330A5000630A600051E192B2E
:10062000851DBC0A851D242B051DBC03051D242B1F
:10063000262BA40B212BA50B212BA60B212BB30AB8
:10064000242B051E192BA80A2714272B27108830C6
:10065000A000C730A1000230A200A00B2D2BA10BDF
:100660002D2BA20B2D2B0800A001E130A1005A3048
:10067000A200861C402BA10B392BA20B392B792B06
:10068000A130A1002330A200A10B442BA20B442BCC
:10069000FA30A1007530A200861C532BA10B4C2B05
:1006A000A20B4C2B792B8B30A1001230A200A10B96
:1006B000572BA20B572B861CA0166E23861C2016C8
:1006C0006E23861CA0156E23861C20156E23861CA7
:1006D000A0146E23861C20146E23772B4D30A100AE
:1006E0000330A200A10B722BA20B722B0800A714DF
:1006F0007A2BA71003112008103A0319BC0A20080E
:10070000113A0319BC0320082F3A0319BC0A200828
:100710002E3A0319BC032008203A0319A80A20081E
:10072000213A0319A80320081F3A0319A80A200830
:100730001E3A0319A8032008253A0319A801200826
:10074000283A0319A80120080C3A0319B30A200813
:10075000333A0319B30A20080D3A0319B10A2008E5
:10076000323A0319B10A0800D7233008403E4C2220
:1007700029083F3C4C228625271D08002B08613E96
:100780004C222C08703E4C222D08803E2F074C2214
:100790002D08B03C2F074C222F08D03C2E074C22AE
:1007A0002F08FF3CA0002E0820024C2208003E2209
:1007B00088304C22080044304C22080083169A00EE
:1007C0008312200883169B001C1555309D00AA300B
:1007D0009D009C149C18EA2B1C118C138312A00AF8
:1007E0000800200883169B001C141A088312A00A14
:1007F0000800A001F123A900F123AB00F123AC0014
:10080000F123AD00F123AE00F123AF00F123B000DE
:10081000F123B2000800A0012908DE232B08DE2303
:100820002C08DE232D08DE232E08DE232F08DE23EE
:100830003008DE233208DE2308002908AA00A901B7
:10084000290803112A06031908002908BC00CD2035
:100850009722E8228E30612001233C08A000BD01D0
:1008600003140430A002031C372CBD0A312C0311E1
:10087000BD080319432C3D08BF3E86133120FF30CD
:100880003120BD0B372CB423A90A5530A000A3306A
:10089000A100A00B492CA10B492C202C6224CC30A8
:1008A000772444307724FA30A000A00B552C622422
:1008B000CC307724BE3077248624BE008624BF0047
:1008C000932408006E247224A030A000A00B662C94
:1008D0006E246430A000A00B6B2C08008316051753
:1008E0008312080083160513831205130800A10064
:1008F0000830A200A10C722403186E240A30A00054
:10090000A00B802C6E24A20B7A2C08000830A200C9
:10091000A1016E2472246E24051B0314A10CA20BEA
:10092000892C2108080003013F19403EBF18203ED2
:100930003F18103EBE1B083E3E1B043EBE1A023E40
:100940003E1A013EA0000301BE19323E3E19193E77
:10095000BE180C3E3E18063EBE002008BF00080030
:100960002808083A031DC42C8C3061204E243F080F
:10097000A000EA2201232C3031203E08A000EA2208
:1009800025086420312008004E2403143F08320259
:100990008517031885130800BF30612049303120C6
:1009A0004430312008232718D22C3423A718D22C06
:1009B0004030A000F123B400F123B5000311B408C6
:1009C000031DF52CB408031DF52CB40FEA2CB50F4C
:1009D000EA2CE52C051EEF2C861CEF2CE52C403074
:1009E000A0003408DE233508DE233408A000EA2204
:1009F000FE223508A000EA22FE223A303120BC0156
:100A0000A801B601B701B801B901BA01BB01C930EB
:100A100061203608162537081625380816253908A6
:100A200016253A0816253B0816251A2DA000EA229D
:100A300004230800A92203113C08003A03193925B0
:100A40003C08013A03193D253C08023A03194125A7
:100A50003C08033A031945253C08043A0319492583
:100A60003C08053A03194D253C08063A0319572D51
:100A7000072D36085125B600080037085125B70064
:100A8000080038085125B800080039085125B90078
:100A900008003A085125BA0008003B085125BB0060
:100AA0000800A80042267B26AE22280808007B25E5
:100AB0007B257B253508A000EA220311360826068F
:100AC000031D802D37082506031D802D38082406B8
:100AD000031D802D3408A000EA22031139082606E0
:100AE000031D802D3A082506031D802D3B08240692
:100AF000031D802D812D340CB40C350DB50D08006F
:100B000008005730A0004830DE2308005730A0000E
:100B1000F123B40003113408483A271103192715AB
:100B20000800D0304C220800D1304C220800D030D0
:100B3000832208009725271E0800BC01A225A725AF
:100B4000AA25E72D3E22912503014C22080003012E
:100B50004C2208003E22912503014C223E2294257E
:100B600060226D22C00060226D22C10060226D22D1
:100B7000C20060226D22C30060226D22C400602288
:100B80006D22C50060227422C6004008D825C0002E
:100B90004108D825C1004208D825C2004408D825FC
:100BA000C4004508D825C5004608D825C600080059
:100BB000A000200E0F39A10020080F39A000A10AC3
:100BC000A10BE42D200808000A30A007E02D7B26A9
:100BD000BF306120420801263A3031204108012609
:100BE00020303120440801262E30312045080126CE
:100BF0002E3031203230312030303120460801266D
:100C0000052EA000EA2201230800A92203113C08B6
:100C1000003A03191F2E3C08013A0319262E3C08FE
:100C2000023A03192D2E3C08033A0319342E3C08CE
:100C3000043A03193B2E3C08053A0319532E420887
:100C4000A8004226B4222808C200E72D4108A800C7
:100C50004226BA222808C100E72D4408A8004226EF
:100C6000C0222808C400E72D4508A8004226C62255
:100C70002808C500E72D4608A8004226CC222808EF
:100C8000C600E72D4E26082327184E2627180800F1
:100C90004E263423A7180800C424422E28083C02FC
:100CA000A807BC02080042086326C2004108632668
:100CB000C10044086326C40045086326C5004608F1
:100CC0006326C6006B2EA000EA222508A000A00E15
:100CD0002408200708003E22912501304C224108BB
:100CE0004C2242084C224C2244084C2245084C22FB
:100CF00046084C2208008F306120DC3031206530FE
:100D0000A0006230A100A00B832EA10B832E8F3098
:100D100061202030312008000614B301B101A80180
:100D200085130C20F92386252719A32E8F20BE308A
:100D3000A0004B30A1001530A200A00B9D2EA10BEE
:100D40009D2EA20B9D2ED7239F3E4C22BF3E4C22B0
:100D5000DF3E4C22FF3E4C226F3E4C227F3E4C2217
:100D60001D24B42375278E2703112808003A031980
:100D7000DF2E2808013A0319F52E2808023A031934
:100D8000FC2E2808033A03190D2F2808043A0319EA
:100D9000142F2808053A03191B2F2808063A0319AF
:100DA0003E2F2808073A03194B2F2808083A031941
:100DB0005C2F2808093A03196D2FA80AB12E2908BB
:100DC000BC00CD209722E8228E30612001233C0810
:100DD000A000BD0103140430A002031CF12EBD0AC3
:100DE000EB2EA1273C08A900B12E2B08BC00E12066
:100DF000EF200327AB00B12E2C08BC00E120FE2021
:100E00000327AC00B12E9D22E8228E306120012301
:100E10003C08BD00A1273C0808002D08BC000F219C
:100E20001F212127AD00B12E2E08BC000F21322139
:100E30002127AE00B12E2F08BC0041212127AF0091
:100E4000B12E9D223C08BD00103EA1002108BF3EEE
:100E500086133120FF303120A10B262F03113D08CE
:100E6000103A0319BD033D08BF3E86133120C83038
:100E70003120C9303120AD273C0808003008BC00C3
:100E80005521A322E8228F306120A40A0423AD2734
:100E90003C08B000B12EDE213208BC00B4249122FF
:100EA000E822CC30612001232C3031203030312039
:100EB000AD273C08B200B12EBC019D21B7213C1CDE
:100EC000D7213C18D02108233423281C5D2F3C1C3B
:100ED000B12E9A250930A800B12E8625A801271920
:100EE000B12E0C22CC24A801B12E3318782F080083
:100EF000331C892F0610D723DB232A229725271E90
:100F0000852FC4306120AA25DE2708233423C4247A
:100F1000782F06141D243110A80108003118912FD4
:100F20000800311C9D2F3318782FD723DB236D2128
:100F30008A2108233423C424912F1D243110A801B1
:100F400008000311BD080319AD2F3D08BF3E8613ED
:100F50003120FF303120BD0BA12F1930A300082311
:100F6000271808003423A7180800B024C424A30BB2
:100F7000AF2F0B24A8019725271E08000823271848
:100F800008003423A71808005220AA254408012687
:100F90002E303120450801262E303120460801260A
:100FA0008C3061205430312065303120BC3031200C
:100FB000BE303120C0306120DE27E92F42080126F3
:100FC0003A303120410801263A30312040080126CC
:0C0FD0000800CC306120C424B724BE2FE0
:02400E00703F01
:10420000080008000800080008000800000023005B
:10421000360023004E0062002A00390062001800B8
:1042200030004B0016002D005700170000002E0034
:1042300024000400350053001D005D0044001C00F4
:104240005E005D005E002000050038001A005F007F
:104250005F0027001700540049002D000A001800D5
:10426000250049004B002B000A004B002E001B00CC
:104270001D0043002D004900300001001000220005
:10428000000000001B000D0009003500150027008C
:1042900057004E004F00480000004B00200009006E
:1042A0002300200015002B00360005005D00CD0026
:1042B0002E001800410044002300050019003600BC
:1042C0002D00360000000D002A0057006300520048
:0442D0002D000A00B3
:00000001FF
